:02000000052ACF
:080008000B19892A8B18932AB9
:100010000C189C2A090082073034313432343334CE
:100020003434353436343734383439343034313488
:100030003234333434343534363437343834393474
:100040003034313432343334343435343634373474
:100050003834393430343134323433343434353460
:10006000363437343834393430343134323433344C
:100070003434353436343734383439343034313438
:100080003234333434343534363437343834393424
:100090003034313432343334820730343034303415
:1000A000303430343034303430343034303431342F
:1000B0003134313431343134313431343134313418
:1000C00031343234323432343234323482073034E0
:1000D0003034303430343034303430343034303400
:1000E00030343134313431343134313431343134E9
:1000F00031343134313432343234323432343234D3
:1001000032343234323432343234333433343334BC
:1001100033343334333433343334333433343434A6
:10012000343434343434343434343434343434348F
:100130003434353435343534353435343534353478
:10014000353435343534303400000030B0005E23AF
:10015000B418AE28AB1FAE28AB18B32827084C2024
:10016000A500F724B6282030A500F724B418BC2831
:10017000AB1FBC28AB18C12827080B20A500F7240B
:10018000C4282030A500F724EC24B418CB282B1F5A
:10019000CB28AB18D02828086620A500F724D32840
:1001A0002030A500F724B418D9282B1FD928AB1864
:1001B000DE2828080B20A500F724E1282030A50020
:1001C000F7240230A5001423F4220F230E30A500DB
:1001D0001423F4220F23B418F128AB1EF128AB1816
:1001E000F62829086620A500F724F9282030A50064
:1001F000F724B418FF28AB1EFF28AB1804292908E0
:100200000B20A500F72407292030A500F724851D21
:100210000A292F14B4184129851941292F1C412975
:100220002F10AB1F1829AB132B17AB122B12412920
:100230002B1F1F292B13AB16AB132B1241292B1E7F
:100240002829AB12AB172B132B121E256D22412927
:10025000AB1E4129AB12AB132B132B164322831673
:1002600000309B0083122708DA22831601309B009E
:1002700083122808DA22831602309B008312290891
:10028000DA22B4186E291830270203195829AB1F37
:100290006E29051A5A29B11C4F29AD0B6E29B114CC
:1002A0001830270203195829A70A5030AD006E29CB
:1002B000A7016E29B110851A6D29311D6129AD0B79
:1002C0006E2931150030270203196A29A70350301F
:1002D000AD006E291730A7006E293111B4189B2983
:1002E0003C302802031985292B1F9B29051A8729D1
:1002F000B11D7C29AD0B9B29B1153C302802031997
:100300008529A80A5030AD009B29A8019B29B1116D
:10031000851A9A29311E8E29AD0B9B293116003082
:10032000280203199729A8035030AD009B293B30C0
:10033000A8009B293112B418C8293C30290203199E
:10034000B229AB1EC829051AB429B11EA929AD0BC3
:10035000C829B1163C3029020319B229A90A503024
:10036000AD00C829A901C829B112851AC729311FB2
:10037000BB29AD0BC8293117003029020319C42944
:10038000A9035030AD00C8293B30A900C82931135A
:100390002B1EDF29061CCD29AF160618DF29AF1E3C
:1003A000DF29AF12851CD529DC2934191E2534110B
:1003B0008514B4145122DF290000000000002B1E18
:1003C000E929B41CE929861DE629E9298510B4101C
:1003D0007B22AC0BA528AB1CEF29AB10F029AB148A
:1003E0003730AC00B41F042AB410851005155F2205
:1003F000061CFB29AF160618F829AF1EF8290511AF
:10040000AF124322B4133415A5280301831203133A
:100410008B008C0083168C00831207309F0098019C
:100420009201970183169F01831290010313831297
:10043000850186018316C2308100093086008C3028
:100440009F00F830850000308B0083122030900030
:100450001E258610AA01AB01AB142B163730AC0059
:100460005030AD002830AE000A30B300B410B413E1
:10047000850125230C1083160C14831210140B17FE
:100480008B174322A428861006110830A5001423D8
:10049000F4220F230030A5001423F4220F236B2332
:1004A0000800861006110830A5001423F4220F233B
:1004B0000130A5001423F4220F23D2230800861054
:1004C00006110830A5001423F4220F230030A500E4
:1004D0001423F4220F23112408008610061108307B
:1004E000A5001423F4220F230130A5001423F422C5
:1004F0000F2364240800861006110830A500142379
:10050000F4220F230130A5001423F4220F23AD247D
:100510000800A000030EA10083120B11210E83001E
:10052000A00E200E0900A000030EA1008B10210ECA
:100530008300A00E200E0900A000030EA100000001
:1005400060308E009E308F00B30BD42A0A30B30087
:10055000B41CD42AA903003029020319C92AFF3088
:1005600029020319B42AD42A3B30A900A803FF307A
:1005700028020319BC2AD42A3B30A80000302702E5
:100580000319C32AA7030C10210E8300A00E200E0E
:100590000900003027020319CE2AD42A003028028D
:1005A0000319D32AD42AB4170C10210E8300A00EED
:1005B000200E090083168B131C159A0055309D00E0
:1005C000AA309D009C148B179C18E42A1C119C13C4
:1005D000831208008B1383169B001C141C18EE2A30
:1005E0001A0883128B17080005140000000005107C
:1005F0000800F130A2003430A300A20BFD2AA30BA7
:10060000FD2A000000000800FB30A2000230A30019
:10061000A20B082BA30B082B0000000008003530AC
:10062000A200A20B112B0800A5198617A51D861381
:1006300025190617251D0613A5188616A51C861252
:1006400025180616251C06120800F9220330A500FD
:10065000142386100611F4220F23F922F4220F230B
:10066000F4220F230230A5001423F4220F23F422D6
:100670000F230C30A5001423F4220F230130A50012
:100680001423F4220F230030A5001423F4220F2397
:100690000030A5001423F4220F230130A5001423F9
:1006A000F4220F23F9220030A5001423F4220F2393
:1006B0000C30A5001423F4220F2308008610061125
:1006C0000C30A5001423F4220F233008A5001423B6
:1006D000F4220F230800861406110230A50014230B
:1006E000F4220F230030A5001423F4220F23053039
:1006F000A5001423F4220F230430A5001423F422B0
:100700000F230430A5001423F4220F230130A50089
:100710001423F4220F230B30A5001423F4220F23FB
:100720000930A5001423F4220F230430A50014235C
:10073000F4220F230D30A5001423F4220F230430DC
:10074000A5001423F4220F230530A5001423F4225E
:100750000F230530A5001423F4220F230030A50039
:100760001423F4220F230230A5001423F4220F23B4
:100770000030A5001423F4220F230230A500142317
:10078000F4220F230030A5001423F4220F2302309B
:10079000A5001423F4220F230030A5001423F42213
:1007A0000F230800861406110230A5001423F4223A
:1007B0000F230030A5001423F4220F230430A500DA
:1007C0001423F4220F230330A5001423F4220F2353
:1007D0000A30A5001423F4220F230B30A5001423A4
:1007E000F4220F230430A5001423F4220F23053034
:1007F000A5001423F4220F230530A5001423F422AE
:100800000F230430A5001423F4220F230230A50087
:100810001423F4220F230030A5001423F4220F2305
:100820000800861406110230A5001423F4220F23B9
:100830000030A5001423F4220F230A30A50014234E
:10084000F4220F230130A5001423F4220F230630D5
:10085000A5001423F4220F230F30A5001423F42243
:100860000F230B30A5001423F4220F230F30A50013
:100870001423F4220F230630A5001423F4220F239F
:100880000F30A5001423F4220F230B30A5001423EE
:10089000F4220F230330A5001423F4220F23023087
:1008A000A5001423F4220F230030A5001423F42202
:1008B0000F230230A5001423F4220F230030A500DB
:1008C0001423F4220F230800861406110430A50017
:1008D0001423F4220F230230A5001423F4220F2343
:1008E0000A30A5001423F4220F230E30A500142390
:1008F000F4220F230A30A5001423F4220F23003022
:10090000A5001423F4220F230430A5001423F4229D
:100910000F230F30A5001423F4220F230530A50068
:100920001423F4220F230030A5001423F4220F23F4
:100930000230A5001423F4220F230030A500142355
:10094000F4220F230230A5001423F4220F230030D9
:10095000A5001423F4220F23080086140611023088
:10096000A5001423F4220F230030A5001423F42241
:100970000F230430A5001423F4220F230330A50015
:100980001423F4220F230530A5001423F4220F238F
:100990000430A5001423F4220F230430A5001423EF
:1009A000F4220F230F30A5001423F4220F230A3062
:1009B000A5001423F4220F230830A5001423F422E9
:1009C0000F230230A5001423F4220F230030A500CA
:1009D0001423F4220F2308000330A5001423F4226B
:1009E0000F230A30A5001423F4220F2308008614D5
:1009F0000611A51B8617A51F8613251B0617251F85
:100A00000613A51A8616A51E8612251A0616251E79
:100A10000612F4220F23A5198617A51D8613251982
:100A20000617251D0613A5188616A51C861225185F
:100A30000616251C0612F4220F2308000030EA22B5
:100A4000A7000130EA22A8000230EA22A90008002B
:02400E00013F70
:1042000000000000050000000000000000000000A9
:10421000000001000000000000000000000000009D
:10422000FF00FF00FF00FF00FF00FF00FF00FF0096
:10423000FF00FF00FF00FF00FF00FF00FF00FF0086
:10424000FF00FF00FF00FF00FF00FF00FF00FF0076
:10425000FF00FF00FF00FF00FF00FF00FF00FF0066
:10426000FF00FF00FF00FF00FF00FF00FF00FF0056
:10427000FF00FF00FF00FF00FF00FF00FF00FF0046
:10428000FF00FF00FF00FF00FF00FF00FF00FF0036
:10429000FF00FF00FF00FF00FF00FF00FF00FF0026
:1042A000FF00FF00FF00FF00FF00FF00FF00FF0016
:1042B000FF00FF00FF00FF00FF00FF00FF00FF0006
:1042C000FF00FF00FF00FF00FF00FF00FF00FF00F6
:1042D000FF00FF00FF00FF00FF00FF00FF00FF00E6
:1042E000FF00FF00FF00FF00FF00FF00FF00FF00D6
:1042F000FF00FF00FF00FF00FF00FF00FF00FF00C6
:00000001FF
